
 Start  Stop   Length Name                   Class
 00000H 000ADH 000AEH EXPORTLM_TEXT          CODE
 000AEH 01B4BH 01A9EH CANON_TEXT             CODE
 01B4CH 0240BH 008C0H _TEXT                  CODE
 0240CH 024D7H 000CCH NETLIB                 CODE
 024D8H 02B7DH 006A6H SECURITY_TEXT          CODE
 02B7EH 02B7EH 00000H SSI_TEXT               CODE
 02B7EH 02C0BH 0008EH SERVER_TEXT            CODE
 02C0CH 02C0CH 00000H SRVSTRNG_TEXT          CODE
 02C0CH 02E0DH 00202H WKSTA_TEXT             CODE
 02E0EH 02E0EH 00000H DLLMGMT_TEXT           CODE
 02E0EH 03249H 0043CH MAILSLOT_TEXT          CODE
 0324AH 0343FH 001F6H RPC_TEXT               CODE
 03440H 03441H 00002H REMOTE_TEXT            CODE
 03442H 03569H 00128H UTIL_TEXT              CODE
 0356AH 0358CH 00023H ASMLIB_TEXT            CODE
 0358EH 0358EH 00000H APIMESS_TEXT           CODE
 0358EH 0358EH 00000H DEFALLOC_TEXT          CODE
 0358EH 0358EH 00000H DEFFREE_TEXT           CODE
 0358EH 035EBH 0005EH DEFMEMRT_TEXT          CODE
 035ECH 035ECH 00000H NULLSTR_TEXT           CODE
 035F0H 04887H 01298H APITABLD5_DATA         FAR_DATA
 04888H 04FB3H 0072CH _DATA                  DATA
 04FB4H 0502DH 0007AH STRINGSEGMENT          DATA
 0502EH 0502EH 00000H XIFB                   DATA
 0502EH 05035H 00008H XIF                    DATA
 05036H 05036H 00000H XIFE                   DATA
 05036H 0529AH 00265H CONST                  CONST
 0529CH 0529CH 00000H _BSS                   BSS

 Origin   Group
 0488:0   DGROUP

  Address         Publics by Name

 01B4:0516       Canonicalize
 0344:0000       DEADTABLEENTRY
 02E0:0132       DOSDELETEMAILSLOT
 01B4:0656       DOSICANONICALIZE
 02E0:018E       DOSMAKEMAILSLOT
 02E0:02E4       DOSREADMAILSLOT
 02E0:036E       DOSWRITEMAILSLOT
 0344:0002       I_NETGETCDNAMES
 000A:14E6       I_NETNAMECOMPARE
 000A:000E       I_NETPATHCANONICALIZE
 000A:0932       I_NETPATHTYPE
 01B4:0599       l0_PathSep
 01B4:05A4       l1_SkipBack
 01B4:064C       l2_ScanPathChar
 01B4:0697       l3_PathChrCmp
 01B4:06F0       l4_NameTrans
 01B4:0715       l5_NORMSCAN
 01B4:0762       l6_GetLet
 01B4:079B       l7_SPCHK
 01B4:07A2       l8_PackName
 0344:00B0       MYDOSALLOCSEG
 0344:00EA       MYDOSFREESEG
 0344:0108       MYDOSREALLOCSEG
 024D:0008       NETGETDCNAME
 0324:012A       NETIISREMOTE
 0324:000A       NETIREMOTEAPI
 02C0:000C       NETSERVERENUM2
 02B7:000E       NETSERVERGETINFO
 02C0:00F2       NETWKSTAGETINFO
 01B4:059B       PathSepGotCh
 000A:0116       R_I_NETPATHCANONICALIZE
 024D:00A1       WGETDCNAME
 000A:158A       WI_NETNAMECOMPARE
 000A:0144       WI_NETPATHCANONICALIZE
 000A:09D4       WI_NETPATHTYPE
 02C0:01AA       WWKSTAGETINFO
 0488:069C       _AdminProcess
 0488:06B0       _AdminProcessCount
 0488:06B2       _AdminProcessSem
 0488:0728       _ALLOCATOR
 035F:0000       _APItable
 0488:021C       _basic_api_table
 02E0:000E       _build_mailslot_name
 0488:067E       _Caller_Info
 0000:0063       _CallExport
 0488:00DC       _cbMaxPathCompLen
 0488:00DA       _cbMaxPathLen
 0488:066E       _cname
 0488:0692       _Data_Sem
 01B4:0826       _DoInt
 01B4:082C       _DoIntP
 01B4:0829       _DoIntR
 01B4:082F       _DoIntx
 0488:06B8       _DomainSem
 0000:0000       _DOSDLLInit
 0488:0A1C       _edata
 0488:06FC       _Encrypt_Sem
 0488:0A1C       _end
 0488:0008       _errno
 0000:0046       _ExportInit
 0000:00A4       _FREE
 0488:0730       _FREEMEM
 0000:00A9       _GETENV
 0356:000A       _getenv_addr
 0000:0081       _GetExportTableVersion
 000A:1670       _GetToken
 024D:05FC       _get_temp_ms
 01B4:01EA       _ininlsf
 0488:021A       _is_basic_redir
 0488:06CC       _LogonDCName
 0488:06EC       _LogonDomain
 0000:009F       _MALLOC
 01B4:001C       _memsetf
 0488:0700       _MslotName
 0488:0886       _num_server_info
 0488:06B6       _PinballInstalled
 0488:06BC       _PrimaryDCName
 0488:06DC       _PrimaryDomain
 0488:0696       _RC_Sem
 0356:001E       _rdr_open
 0488:069A       _Reader_Count
 0488:072C       _REALLOCATOR
 01B4:03A4       _strcatf
 01B4:004E       _strchrf
 01B4:0340       _strcmpf
 01B4:036C       _strcpyf
 01B4:018E       _strcspnf
 01B4:0296       _stricmpf
 01B4:0326       _strlenf
 01B4:00DA       _strncpyf
 01B4:007C       _strnicmpf
 01B4:0104       _strrchrf
 01B4:0132       _strspnf
 0240:000C       _strtailf
 01B4:02EC       _struprf
 0488:0014       _theTable
 0488:0892       _txt_REM_connection_info_0
 0488:0894       _txt_REM_connection_info_1
 0488:07F2       _txt_REM_dc_name
 0488:07BE       _txt_REM_I_NetListCanonicalizeP
 0488:07C8       _txt_REM_I_NetNameCanonicalizeP
 0488:07D6       _txt_REM_I_NetNameCompare_P
 0488:07DB       _txt_REM_I_NetNameValidate_P
 0488:07CE       _txt_REM_I_NetPathCanonicalizeP
 0488:07DF       _txt_REM_I_NetPathCompare_P
 0488:07E4       _txt_REM_I_NetPathType_P
 0488:089C       _txt_REM_NetConnectionEnum_P
 0488:07E8       _txt_REM_NetGetDCName_P
 0488:07EC       _txt_REM_NetLogonEnum_P
 0488:07F6       _txt_REM_NetServerAdminCommand_
 0488:07F6       _txt_REM_NetServerAdminCom_P
 0488:08A3       _txt_REM_NetServerDiskEnum_P
 0488:07FF       _txt_REM_NetServerEnum2_P
 0488:0807       _txt_REM_NetServerEnum_P
 0488:0888       _txt_REM_NetServerGetInfo_P
 0488:088D       _txt_REM_NetServerSetInfo_P
 0488:08AC       _txt_REM_NetWkstaGetInfo_P
 0488:0907       _txt_REM_NetWkstaSetInfo_P
 0488:0990       _txt_REM_NetWkstaSetUID_P
 0488:0985       _txt_REM_NetWkstaUserLogoff_P
 0488:097A       _txt_REM_NetWkstaUserLogon_P
 0488:0A1A       _txt_REM_nulstr
 0488:07FD       _txt_REM_server_admin_command
 0488:08A9       _txt_REM_server_diskenum
 0488:080D       _txt_REM_server_info_0
 0488:0811       _txt_REM_server_info_1
 0488:0819       _txt_REM_server_info_2
 0488:084A       _txt_REM_server_info_3
 0488:087E       _txt_REM_server_info_table
 0488:0976       _txt_REM_user_logoff_info_1
 0488:0953       _txt_REM_user_logon_info_0
 0488:0958       _txt_REM_user_logon_info_1
 0488:096D       _txt_REM_user_logon_info_2
 0488:08B1       _txt_REM_wksta_info_0
 0488:090C       _txt_REM_wksta_info_0_setinf
 0488:08D3       _txt_REM_wksta_info_1
 0488:08F8       _txt_REM_wksta_info_10
 0488:092E       _txt_REM_wksta_info_1_setinf
 0488:0900       _txt_REM_WWkstaGetInfo_P
 0488:0658       _uname
 0488:068E       _Writer_Sem
 0000:0000  Abs  __ACRTUSED
 0000:0000  Abs  __ADBUSED
 0000:9876  Abs  __anlsused
 0488:021E       __CollateTable
 01B4:0442       __DOSCASEMAP
 01B4:03EC       __DOSGETCOLLATE
 0488:09CF       __DosMVDMErrorMsg
 01B4:07D8       __DosVersionCheck
 0000:0001  Abs  __DosVersionCheckInit
 0488:0998       __DosVersionCheckMsg
 0488:0A1C       __edata
 0488:0A1C       __end
 0488:0A19       __InMVDMBox
 0488:0012       __rpc_hostDS
 0488:041E       __ToLowerCaseTable
 0488:031E       __ToUpperCaseTable
 0358:000E       ___default_allocator
 0358:0042       ___default_available
 0358:005A       ___default_freemem
 0358:002A       ___default_reallocator
 01B4:08AE       ___segread
 0488:051E       ____ctype
 0488:051E       ____ctype_

  Address         Publics by Value

 0000:0000  Abs  __ACRTUSED
 0000:0000  Abs  __ADBUSED
 0000:0000       _DOSDLLInit
 0000:0001  Abs  __DosVersionCheckInit
 0000:0046       _ExportInit
 0000:0063       _CallExport
 0000:0081       _GetExportTableVersion
 0000:009F       _MALLOC
 0000:00A4       _FREE
 0000:00A9       _GETENV
 000A:000E       I_NETPATHCANONICALIZE
 000A:0116       R_I_NETPATHCANONICALIZE
 000A:0144       WI_NETPATHCANONICALIZE
 000A:0932       I_NETPATHTYPE
 000A:09D4       WI_NETPATHTYPE
 000A:14E6       I_NETNAMECOMPARE
 000A:158A       WI_NETNAMECOMPARE
 000A:1670       _GetToken
 01B4:001C       _memsetf
 01B4:004E       _strchrf
 01B4:007C       _strnicmpf
 01B4:00DA       _strncpyf
 01B4:0104       _strrchrf
 01B4:0132       _strspnf
 01B4:018E       _strcspnf
 01B4:01EA       _ininlsf
 01B4:0296       _stricmpf
 01B4:02EC       _struprf
 01B4:0326       _strlenf
 01B4:0340       _strcmpf
 01B4:036C       _strcpyf
 01B4:03A4       _strcatf
 01B4:03EC       __DOSGETCOLLATE
 01B4:0442       __DOSCASEMAP
 01B4:0516       Canonicalize
 01B4:0599       l0_PathSep
 01B4:059B       PathSepGotCh
 01B4:05A4       l1_SkipBack
 01B4:064C       l2_ScanPathChar
 01B4:0656       DOSICANONICALIZE
 01B4:0697       l3_PathChrCmp
 01B4:06F0       l4_NameTrans
 01B4:0715       l5_NORMSCAN
 01B4:0762       l6_GetLet
 01B4:079B       l7_SPCHK
 01B4:07A2       l8_PackName
 01B4:07D8       __DosVersionCheck
 01B4:0826       _DoInt
 01B4:0829       _DoIntR
 01B4:082C       _DoIntP
 01B4:082F       _DoIntx
 01B4:08AE       ___segread
 0240:000C       _strtailf
 024D:0008       NETGETDCNAME
 024D:00A1       WGETDCNAME
 024D:05FC       _get_temp_ms
 02B7:000E       NETSERVERGETINFO
 02C0:000C       NETSERVERENUM2
 02C0:00F2       NETWKSTAGETINFO
 02C0:01AA       WWKSTAGETINFO
 02E0:000E       _build_mailslot_name
 02E0:0132       DOSDELETEMAILSLOT
 02E0:018E       DOSMAKEMAILSLOT
 02E0:02E4       DOSREADMAILSLOT
 02E0:036E       DOSWRITEMAILSLOT
 0324:000A       NETIREMOTEAPI
 0324:012A       NETIISREMOTE
 0344:0000       DEADTABLEENTRY
 0344:0002       I_NETGETCDNAMES
 0344:00B0       MYDOSALLOCSEG
 0344:00EA       MYDOSFREESEG
 0344:0108       MYDOSREALLOCSEG
 0356:000A       _getenv_addr
 0356:001E       _rdr_open
 0358:000E       ___default_allocator
 0358:002A       ___default_reallocator
 0358:0042       ___default_available
 0358:005A       ___default_freemem
 035F:0000       _APItable
 0488:0008       _errno
 0488:0012       __rpc_hostDS
 0488:0014       _theTable
 0488:00DA       _cbMaxPathLen
 0488:00DC       _cbMaxPathCompLen
 0488:021A       _is_basic_redir
 0488:021C       _basic_api_table
 0488:021E       __CollateTable
 0488:031E       __ToUpperCaseTable
 0488:041E       __ToLowerCaseTable
 0488:051E       ____ctype_
 0488:051E       ____ctype
 0488:0658       _uname
 0488:066E       _cname
 0488:067E       _Caller_Info
 0488:068E       _Writer_Sem
 0488:0692       _Data_Sem
 0488:0696       _RC_Sem
 0488:069A       _Reader_Count
 0488:069C       _AdminProcess
 0488:06B0       _AdminProcessCount
 0488:06B2       _AdminProcessSem
 0488:06B6       _PinballInstalled
 0488:06B8       _DomainSem
 0488:06BC       _PrimaryDCName
 0488:06CC       _LogonDCName
 0488:06DC       _PrimaryDomain
 0488:06EC       _LogonDomain
 0488:06FC       _Encrypt_Sem
 0488:0700       _MslotName
 0488:0728       _ALLOCATOR
 0488:072C       _REALLOCATOR
 0488:0730       _FREEMEM
 0488:07BE       _txt_REM_I_NetListCanonicalizeP
 0488:07C8       _txt_REM_I_NetNameCanonicalizeP
 0488:07CE       _txt_REM_I_NetPathCanonicalizeP
 0488:07D6       _txt_REM_I_NetNameCompare_P
 0488:07DB       _txt_REM_I_NetNameValidate_P
 0488:07DF       _txt_REM_I_NetPathCompare_P
 0488:07E4       _txt_REM_I_NetPathType_P
 0488:07E8       _txt_REM_NetGetDCName_P
 0488:07EC       _txt_REM_NetLogonEnum_P
 0488:07F2       _txt_REM_dc_name
 0488:07F6       _txt_REM_NetServerAdminCommand_
 0488:07F6       _txt_REM_NetServerAdminCom_P
 0488:07FD       _txt_REM_server_admin_command
 0488:07FF       _txt_REM_NetServerEnum2_P
 0488:0807       _txt_REM_NetServerEnum_P
 0488:080D       _txt_REM_server_info_0
 0488:0811       _txt_REM_server_info_1
 0488:0819       _txt_REM_server_info_2
 0488:084A       _txt_REM_server_info_3
 0488:087E       _txt_REM_server_info_table
 0488:0886       _num_server_info
 0488:0888       _txt_REM_NetServerGetInfo_P
 0488:088D       _txt_REM_NetServerSetInfo_P
 0488:0892       _txt_REM_connection_info_0
 0488:0894       _txt_REM_connection_info_1
 0488:089C       _txt_REM_NetConnectionEnum_P
 0488:08A3       _txt_REM_NetServerDiskEnum_P
 0488:08A9       _txt_REM_server_diskenum
 0488:08AC       _txt_REM_NetWkstaGetInfo_P
 0488:08B1       _txt_REM_wksta_info_0
 0488:08D3       _txt_REM_wksta_info_1
 0488:08F8       _txt_REM_wksta_info_10
 0488:0900       _txt_REM_WWkstaGetInfo_P
 0488:0907       _txt_REM_NetWkstaSetInfo_P
 0488:090C       _txt_REM_wksta_info_0_setinf
 0488:092E       _txt_REM_wksta_info_1_setinf
 0488:0953       _txt_REM_user_logon_info_0
 0488:0958       _txt_REM_user_logon_info_1
 0488:096D       _txt_REM_user_logon_info_2
 0488:0976       _txt_REM_user_logoff_info_1
 0488:097A       _txt_REM_NetWkstaUserLogon_P
 0488:0985       _txt_REM_NetWkstaUserLogoff_P
 0488:0990       _txt_REM_NetWkstaSetUID_P
 0488:0998       __DosVersionCheckMsg
 0488:09CF       __DosMVDMErrorMsg
 0488:0A19       __InMVDMBox
 0488:0A1A       _txt_REM_nulstr
 0488:0A1C       __end
 0488:0A1C       _edata
 0488:0A1C       __edata
 0488:0A1C       _end
 0000:9876  Abs  __anlsused

Program entry point at 0000:0000
